:10000000DB28A8008417800484138E010C1C8E004A
:1000100023200319D62823200319D6282320D628E5
:10002000A80059200C080D040319D628D0208413E9
:100030002808800664001C281D288C0A03198D0FCF
:100040001A288006D62828088E0601308C008D01DB
:10005000000828050E06031D08008C0A03198D0FE1
:10006000282808008F002A08840028095A208413B1
:100070008F080319D628F03091000E0880389000C0
:10008000F03091030319910003198F030319D62847
:1000900049285D2003010C1828088E1F28088E08A7
:1000A00003190301900F562880063D2857280000A9
:1000B0004028FF3A84178005D6280D080C04031940
:1000C0008C0A80300C1A8D060C198D068C188D0642
:1000D0000D0D8C0D8D0DD6288F018E00FF308E07F3
:1000E000031C8F07031CD62803308D00DF307A20D5
:1000F0006E288D01E83E8C008D09FC30031C83289E
:100100008C07031880288C0764008D0F80280C183A
:1001100089288C1C8D2800008D2808008D018F01F6
:100120008E000230A0288E000330A0288D018F01A0
:100130008E000130A0288D018F018E000430A02890
:1001400094000F080D02031DA7280E080C020430AE
:1001500003180130031902301405031DFF30D6289F
:100160000404031DFF30D628910190011030920045
:100170000D0D900D910D0E0890020F08031C0F0F2E
:1001800091020318CA280E0890070F0803180F0FD2
:10019000910703108C0D8D0D920BB8280C08D628F2
:1001A0008C098D098C0A03198D0A08008313031327
:1001B000831264000800831603308500083086002F
:1001C0008312061183160611831286108316861079
:1001D000831206108316061006308312AA00103010
:1001E000A80064308E000A30322032308E00053094
:1001F000322046308E000A30322032308E000230FB
:10020000322001308C0005308400013001200C08C0
:10021000B00001308C0005308400023001200C0851
:10022000B10030088C009B3096209E0030088C0076
:1002300091309B20A0001E0884002008B020A00060
:10024000A10031088C009B309620A20031088C0060
:1002500091309B20A400220884002408B020A40030
:10026000A50020082104840024082504B020A4004F
:10027000A500640024082504031947290630AA00B4
:100280001030A80064308E00053032200129013082
:100290008C0005308400013001200C08B0000130D2
:1002A0008C0005308400023001200C08B1003008B9
:1002B0008C0000308E209E0031088C0000308E2093
:1002C000A0001E0884002008B020A000A100640047
:1002D0002008210403196D2901296400B530310279
:1002E000031C7329B4216400783031020318792982
:1002F000C52164007830300203187F29E7216400AB
:10030000B5303002031C8529D621F8212C088C0039
:100310002D088D008F0106309320031DB32986140C
:100320008316861083120614831606100630831275
:10033000AA001030A80050308E000A3032206430FD
:100340008E00053032206E308E00023032205A305E
:100350008E0002303220861083168610831206101B
:100360008316061083124729AA30B4001722A03042
:10037000B300A030B50017226430B40017227830E3
:10038000B3007830B50017220800AA30B400172255
:100390007830B3007830B50017226430B4001722EB
:1003A000A030B300A030B50017220800AA30B40076
:1003B00017227830B300A030B50017226430B400A3
:1003C0001722A030B3007830B50017220800AA30F9
:1003D000B4001722A030B3007830B5001722643083
:1003E000B40017227830B300A030B50017220800FF
:1003F00001308C008D010630840004301020013063
:100400008C0006308400083001200C08AE000D0876
:10041000AF002E088C002F088D000F308E008F014A
:10042000B420AC000D08AD0001306C200800013094
:10043000B60064000B3036020318372A34088C00EB
:100440008D01063084008030102033088C008D012F
:10045000063084004030102035088C008D010630B5
:100460008400203010200D306C20B60F192A0800AF
:040470006300382AC3
:02400E00F53F7C
:00000001FF
